:100000000C945B0E0C94830E0C94830E0C94830E54
:100010000C94830E0C94830E0C94830E0C94830E1C
:100020000C94830E0C94830E0C94E1180C945319C9
:100030000C94830E0C94830E0C94830E0C94830EFC
:100040000C94830E0C942A150C94830E0C94830E3E
:100050000C94830E0C94830E0C94830E0C943D141C
:100060000C94830E0C94830E0C94830E0C94830ECC
:100070000C94830E0C94830E0C94830E0C94830EBC
:100080000C94C8150C94830E0C94830E0C94830E60
:100090000C94830E0C94830E0C94830E0C94830E9C
:1000A0000C94830E0C94830E0C94830EF712FA12A8
:1000B000E912ED12F1121B131B131B13FE12021394
:1000C00006130C1310131B131613921397139C1380
:1000D000A613B013FA13FA13FA13BA13C413CE13F8
:1000E000D813E513FA13ED13F0F89C8E8783878EEF
:1000F0009CF8F00000FEFF0303030303070EFCF867
:100100000000FEFF0303030303070EFCF80000FFDB
:10011000FF00000000000000FFFF0000FEFF8383DF
:10012000838383C7EE7C380000F8FC0E07030303CB
:10013000070EFCF800003F7FE0C08080C0E07F3FFA
:10014000FFFF01010101010101FFFF0000FFFF0CA2
:100150000C0C0C1C3E77E3C100007FFFC0C0C0C088
:10016000C0E0703F1F00001F3F70E0C0C0C0E070E3
:100170003F1F00007FFFC1C1C1C1C1E3773E1C002A
:10018000001F3F70E0C0C0C0E0703F1F00000000D3
:100190000001FFFF01000000000000002400270014
:1001A0002A002D003000D5F08D14A1C881CFD9F1DF
:1001B000AF20001402130212021502070208020403
:1001C000010C01060100000000808000708804C45A
:1001D00084C48201E21C0000000000000000000056
:1001E00006091516EA19C9D5BC0B325191122B2AF2
:1001F00024140800000000000000000000000001BE
:100200001E22555340504C330000000000000000F7
:1002100000000000000000000000000000000000DE
:1002200000000000000000000000000000000000CE
:10023000000000000070F83878387CFE1C000000D8
:10024000000000000000000000060A0905E6362A4A
:1002500043F4CD8E0E0D14141808000000000000A9
:100260000000000000000000011D2A2C3F2F330079
:10027000000000000000000000000000000000007E
:10028000000000000000000000000000000000006E
:1002900000000000000000708804C484C48201E2F1
:1002A0001C00000000000000000000000000000032
:1002B000001CE31423AA8901AE49300000000000AD
:1002C000000000000000000000000C12090A011EDE
:1002D000000B0807180000000000000000000000EC
:1002E000000000000000000000000000000000000E
:1002F00000000000000000000000000000000000FE
:1003000070F83878387CFE1C000000000000000007
:10031000000000000000000000001CEBDC5576FE31
:10032000513000000000000000000000000000004C
:100330000000000C16151E011F1417180000000005
:1003400000000000000000000000000000000000AD
:10035000000000000000000000000000000000009D
:10036000000000000000000000000000000000008D
:10037000000000000000000000000000000000007D
:10038000000000000000000000000000000000006D
:1003900000000000000040404040404040404440D9
:1003A0004040404040404440404040404040404049
:1003B000404040404040404040404040404040403D
:1003C000000000000000FF1FDFDFDFDFDFDFDFDF17
:1003D000DFDFDFDF1FFF1FDFDFDFDFDFDFDFDFDF8D
:1003E000DFDFDF00FFFF7F7F7F7F7F7F7FFF00FFFB
:1003F000FF0000000000FFE0EEEEEEEEEEEEEEEEAF
:10040000EEEEEEEEE0FFE0EEEEEEEEEEEEEEEEEE17
:10041000EEEEEE00FFFF80B7B7B7B7B780FF00FF83
:10042000FF000000000004040404040404040404A5
:10043000040404040404040404040404040404047C
:1004400004040400FFFFFFFFFFFFFFFFFFFF0004A6
:1004500004000000000080C0F070000808080808D0
:1004600008080808080808080070F0C08080C0F07C
:100470007000303037373737373737373737100076
:10048000000000000000000000000000000000006C
:100490008088D0E080808080808080808040404064
:1004A00040404040602000000000000000000000CC
:1004B000000000000000BCBCBCBCBCBCBEBEB9BDE2
:1004C000BCBCBCBCBFBEB8BCBFB8BCBCBCBCBCBC6C
:1004D000BCBCBCBCBCBCBCBCBCBCBCBCBCBCBCBC5C
:1004E000FCF80000000000E0202020202020202038
:1004F00020202020E000E02020202020202020209C
:10050000202020FF00008080808080808000FF000D
:1005100000FF00000000001F111111111111111135
:10052000111111111F001F111111111111111111B0
:10053000111111FF00007F48484848487F00FF0024
:1005400000FFE0000080FBFBFBFBFBFBFBFBFBFB7E
:10055000FBFBFBFBFBFBFBFBFBFBFBFBFBFBFBFBEB
:10056000FBFBFBFF00000000000000000000FFFBA1
:10057000FBFF3F1F061F7F3F0F8F7F377777777710
:1005800077777777777777377F8F0F3F7F7F3F0F4B
:100590008F7F4F4F484848484848484848486F7FF1
:1005A0003F1F0000000000000000000000000000ED
:1005B000000000000000000000000000000000003B
:1005C000000000000000000000000000000000002B
:1005D000000000000000404040404040404040409B
:1005E000404040404040404040404040404040400B
:1005F00040404040404040404040404040404040FB
:100600004040404040401FDFDFDFDFDFDFDFDFDF74
:10061000DFDF1FFF1FDFDFDFDFDFDFDFDFDFDFDF4A
:10062000DFDFDFDFDFDF1FFF1FDFDFDFDFDFDFDF3A
:10063000DFDFDFDFDF1FE0EEEEEEEEEEEEEEEEEE02
:10064000EEEEE0FFE0EEEEEEEEEEEEEEEEEEEEEED5
:10065000EEEEEEEEEEEEE0FFE0EEEEEEEEEEEEEEC5
:10066000EEEEEEEEEEE004040404040404040404DC
:10067000040404040404040404040404040404043A
:10068000040404040404040404040404040404042A
:1006900004040404040480C0F07000000000001092
:1006A000101010101010101010101010101010104A
:1006B000101010101010101010101010100000006A
:1006C000000070F0C080000000000000000000008A
:1006D000000000000000000000000000000000001A
:1006E000000000000000000000000000000000000A
:1006F000000000000000BCBCBCBCBCBCBCBCBCBCA2
:10070000BCBCBCBCBCBCBCBCBCBCBCBCBCBCBCBC29
:10071000BCBCBCBCBCBCBCBCBCBCBCBCBCBCBCBC19
:10072000BCBCBCBCBCBCE020202020202020202061
:100730002020E000E0202020202020202020202059
:10074000202020202020E000E02020202020202049
:100750002020202020E01F11111111111111111161
:1007600011111F001F11111111111111111111116E
:100770001111111111111F001F111111111111115E
:1007800011111111111FFBFBFBFBFBFBFBFBFBFB27
:10079000FBFBFBFBFBFBFBFBFBFBFBFBFBFBFBFBA9
:1007A000FBFBFBFBFBFBFBFBFBFBFBFBFBFBFBFB99
:1007B000FBFBFBFBFBFB7F3F0F8F7F3F7F7F7F6F51
:1007C0006F6F6F6F6F6F6F6F6F6F6F6F6F6F6F6F39
:1007D0006F6F6F6F6F6F6F6F6F6F6F6F6F7F7F7FF9
:1007E0003F7F8F0F3F7F00000000000000000000EF
:1007F00000000000000000000000000000000000F9
:1008000000000000000000000000000000000000E8
:1008100000000000000000000000000040404040D8
:1008200040404040404040404040404040404040C8
:1008300040404040404040404040404040404040B8
:100840004040404040400000000000FFFF00FF7FAC
:100850007F7F7F7F7F7FFFFF00DFDFDFDFDFDFDF87
:10086000DFDFDFDFDF1FFF1FDFDFDFDFDFDFDFDFF8
:10087000DFDFDFDF1FFF0000000000FFFF00FF8061
:10088000B7B7B7B7B780FFFF00EEEEEEEEEEEEEED5
:10089000EEEEEEEEEEE0FFE0EEEEEEEEEEEEEEEE83
:1008A000EEEEEEEEE0FF0000000000040400FFFFAB
:1008B000FFFFFFFFFFFFFFFF000404040404040424
:1008C00004040404040404040404040404040404E8
:1008D0000404040404040000000000000010373782
:1008E000373737373737373730300070F0C08080D0
:1008F000C0F0700008080808080808080808080878
:10090000080070F0C080000000000000000000003F
:1009100000000000000000000000000000000000D7
:1009200000000000000000000000000000000000C7
:1009300000000000000000000000F8FCBCBCBCBCD3
:10094000BCBCBCBCBCBCBCBCBCBCBCBCBCBCBCBCE7
:10095000BCBCBCBCBCBCBCBCBCBCBCBCBCBCBCBCD7
:10096000BCBCBCBCBCBC00000000FF0000FF0080A1
:100970008080808080800000FF2020202020202098
:100980002020202020E000E0202020202020202007
:1009900020202020E000800000E0FF0000FF007F1A
:1009A00048484848487F0000FF11111111111111EA
:1009B00011111111111F001F11111111111111111C
:1009C000111111111F001F061F3FFFFBFBFF00004D
:1009D0000000000000000000FFFBFBFBFBFBFBFB3B
:1009E000FBFBFBFBFBFBFBFBFBFBFBFBFBFBFBFB57
:1009F000FBFBFBFBFBFB000000001F3F7F6F484839
:100A000048484848484848484F4F7F8F0F3F7F7FAE
:100A10003F0F8F7F37777777777777777777777726
:100A2000377F8F0F3F7F00000000000000000000B4
:100A300000000000000000000000000000000000B6
:100A400000000000000000000000000000000000A6
:100A50000000000000004040404040404044404012
:100A60004040404040444040404040404040404082
:100A700040404040404040404040404040404000B6
:100A8000000000000000DFDFDFDFDFDFDFDFDF1F70
:100A9000FF1FDFDFDFDFDFDFDFDFDFDFDFDF1FFFA6
:100AA000FFFF00FFFF7F7F7F7F7F7F7FFF00FFFFD4
:100AB000000000000000EEEEEEEEEEEEEEEEEEE0F8
:100AC000FFE0EEEEEEEEEEEEEEEEEEEEEEEEE0FF40
:100AD000FFFF00FFFF80B7B7B7B7B780FF00FFFF8A
:100AE00000000000000004040404040404040404DE
:100AF00004040404040404040404040404040404B6
:100B0000040400FFFFFFFFFFFFFFFFFFFF000404DF
:100B1000000000000000C0F0700008080808080885
:100B2000080808080808080070F0C08080C0F0704D
:100B3000003030373737373737373737371000001F
:100B40000000000000000000000000000000008025
:100B500088D0E080808080808080808040404040DD
:100B60004040406020000000000000000000000045
:100B7000000000000000BCBCBCBCBCBEBEB9BDBC1B
:100B8000BCBCBCBFBEB8BCBFB8BCBCBCBCBCBCBCA5
:100B9000BCBCBCBCBCBCBCBCBCBCBCBCBCBCBCFC55
:100BA000F80000000000202020202020202020E04D
:100BB00000E0202020202020202020202020E000F5
:100BC0000000FF00008080808080808000FF0000A7
:100BD000FF00000000001111111111111111111F5E
:100BE000001F1111111111111111111111111F00FB
:100BF0000000FF00007F48484848487F00FF000091
:100C0000FFE000008000FBFBFBFBFBFBFBFBFBFBB7
:100C1000FBFBFBFBFBFBFBFBFBFBFBFBFBFBFBFB24
:100C2000FBFBFF00000000000000000000FFFBFBDA
:100C3000FF3F1F061F003F0F8F7F3777777777774C
:100C4000777777777777377F8F0F3F7F7F3F0F8F6C
:100C50007F4F4F484848484848484848486F7F3F7A
:100C60001F00000000000000000000000000000065
:100C70000000000000000000000000000000000074
:100C80000000000000000000000000000000000064
:100C900000000000000040404040404040404040D4
:100CA0004040404040404040404040404040404044
:100CB0004040404040404040404040404040404034
:100CC000404040404040DFDFDFDFDFDFDFDFDFDFEE
:100CD000DFDF1FFF1FDFDFDFDFDFDFDFDFDFDFDF84
:100CE000DF1FFF1FDFDFDFDFDFDFDFDFDFDFDFDF74
:100CF0001FFF1FDFDFDFEEEEEEEEEEEEEEEEEEEECE
:100D0000EEEEE0FFE0EEEEEEEEEEEEEEEEEEEEEE0E
:100D1000EEE0FFE0EEEEEEEEEEEEEEEEEEEEEEEEFE
:100D2000E0FFE0EEEEEE0404040404040404040412
:100D30000404040404040404040404040404040473
:100D40000404040404040404040404040404040463
:100D5000040404040404080808080808080808082B
:100D60000070F0C08080C0F0700000000000101023
:100D700010101010101010101010101000000000B3
:100D80000070F0C080800000000000000000000043
:100D90000000000000000000000000000000000053
:100DA0000000000000000000000000000000000043
:100DB000000000000000BCBCBCBCBCBCBCBCBCBCDB
:100DC000BCBCBCBCBCBCBCBCBCBCBCBCBCBCBCBC63
:100DD000BCBCBCBCBCBCBCBCBCBCBCBCBCBCBCBC53
:100DE000BCBCBCBCBCBC202020202020202020205B
:100DF0002020E000E0202020202020202020202093
:100E000020E000E020202020202020202020202082
:100E1000E000E02020201111111111111111111108
:100E200011111F001F1111111111111111111111A7
:100E3000111F001F11111111111111111111111197
:100E40001F001F111111FBFBFBFBFBFBFBFBFBFB63
:100E5000FBFBFBFBFBFBFBFBFBFBFBFBFBFBFBFBE2
:100E6000FBFBFBFBFBFBFBFBFBFBFBFBFBFBFBFBD2
:100E7000FBFBFBFBFBFB777777777777777777372A
:100E80007F8F0F3F7F7F3F0F8F7F3F7F7F7F6F6F12
:100E90006F6F6F6F6F6F6F6F6F6F6F6F7F7F7F7F22
:100EA0007F8F0F3F7F7F00000000000000000000E8
:100EB0000000000000000000000000000000000032
:100EC0000000000000000000000000000000000022
:100ED0000000000000000000000000000000000012
:100EE0000000000000000000000000000000000002
:100EF0000040404040404040404040404040404032
:100F00004040404040400000000000000000000061
:100F10000000000000008080C0C0E0E0E0E0E0F001
:100F200000F0F8FF7FBFBFBFBFBFBF7FFFFFFFFF66
:100F300000FFFFFFFF1F0080E0F8FCFEFEFEFEFE4C
:100F4000FEFFFFFFFFFFFFFFFFFFFFFFFFFFFFFFB2
:100F500000FFFF00FFF3EDEDEDEDF3FF00FFFFFFFE
:100F600000FFFFFFFFE0007FFFFFFFFFFFFFFFF736
:100F7000F7F7F7F7F3F3FFFFFFFFFF7F7F7FFFFF39
:100F800000FFFF003F1F1F1F1F1F1F3F001F8FC7B6
:100F90006031180C0404000000000101010101018E
:100FA00001010101010101010101010000000141F4
:100FB0002013070404040404040070F4C48381C0F3
:100FC000F0700008080800000000000000000000A9
:100FD0000000000000000000000000000000000011
:100FE0000000000000000000000000000000000001
:100FF00000000000000000000000000000000000F1
:101000000000000000008080C0C0E0E0F0F0F0F0E0
:10101000F838B8BCBCBCBCBCBCBCBCBCBCBCBCBC5C
:10102000BCBCBCBCBCBC00000000000080C0E0F048
:10103000F8FCFEFEFFFF7F7F3F3F1F1F1F1F1F0F9C
:10104000F70807008040404040404080000000001A
:10105000FF00000000E080601804020101010101AE
:10106000010000000000000000000000000000007F
:10107000FF0000FF000C121212120C00FF00000013
:10108000FF000000001F7F8000000000000000083B
:10109000080808080C0C0000000000808080000098
:1010A000FF0000FFC0E0E0E0E0E0E0C0FFE07038FB
:1010B0009FCEE7F3FBFB0000010102C2E2F2FAFE61
:1010C000FEFEFEFEFEFEFEFEFEFEFEFFFFFFFEBE7D
:1010D000DFECF8FB7B3B1B0B0B7F8F0B3B7C7E3FDE
:1010E0000F8F7F377777DFEFC7B35F7F5F9FA7D71C
:1010F000EFF7EFEFEFE7D3DFDFDFEFD3DFAFBFBF18
:10110000BFDFBBC7EFDFEFDFE7DFE3F7EFDFEFC7FF
:10111000B35F7F5F9FA7B7B7B7B7B7B73797A78753
:10112000A787A79737B7B7B7B7B7B7B7B7B7B7B73F
:10113000B7B7B7B7B7B7B7B7B73797A787A787A76F
:101140009737B7B7B7B7F4FBF7F7F7F4F8FBFBFB44
:10115000FDFBF5E9E0D7DFD7ECF1FBF7FBFDF8F796
:10116000F9F7FBF7FBF1EEF7EFE8EBEBF3F0FBF34E
:10117000F3F0F4F9FBFB0F0F0F0F0F0F0F0F0F0F13
:101180000F0F0F0F0F0F0F0F0F0F0F0F0F0F0F0F6F
:101190000F0F0F0F0F0F0F0F0F0F0F0F0F0F0F0F5F
:1011A0000F0F0F0F0F0F20202020202020436F6DE6
:1011B000706C6574650A0A416C6C20686967682008
:1011C00073636F726520646174610A77617320656F
:1011D00072617365642E2E2E002020202020202096
:1011E000436F6E74726F6C730A0A202020202041B6
:1011F0003A204A756D70206F66660A5570202B2064
:10120000423A2044656C6574652064617461002015
:1012100020202020496E737472756374696F6E7339
:101220000A0A41766F696420746865207472616986
:101230006E21205468650A636C6F7365722069744F
:10124000206765747320746F20796F752C0A746839
:1012500065206D6F726520706F696E747320796F91
:10126000750A77696C6C207261636B207570210060
:1012700000F884722A7284F8000004F870200000DC
:101280000001020505050201000001000000000048
:10129000000000000000000000000000000000004E
:1012A000000000000000000000000000000000003E
:1012B000000000000000000000000000000000002E
:1012C000F0E080000000003EFEFCC000000000F8DE
:1012D000F8F8F0E0C08000F0F0F00000000000003E
:1012E00000000000000000000000000000000000FE
:1012F000071F3FBE380000001F3F3F0000000001F5
:101300007F7F3F03070F3F7F7F7F000000000000CB
:1013100000000000000000000000000000000000CD
:10132000FCF8F0000000C0F0F8783C1C1C9C9CBC51
:10133000F8B800000000FCFCFCCCCCECECECEC0CB5
:10134000000000000000000000000000000000009D
:101350007F3F070000003F3F7F707071733B3B3F52
:101360001F0F000000081F1F1F1C1C1C0C0C0C0C66
:10137000000000000000000000000000000000006D
:10138000000000000000000000000000000000005D
:10139000000000000000000000000000000000004D
:1013A000000000000000000000000000000000003D
:1013B000C0A040A040A0E0408000183838383878FD
:1013C000F8F8F8707060000000E0E0E0E0E0E0E0D5
:1013D000C0C080000000000000008080800000008D
:1013E00000050500050005050005000500040000D6
:1013F000031FFFFEF000000000010FFFFFF8F1F1F6
:10140000F1F3FFFFFE00000000E0FFFFFF1F7EFC86
:10141000898000818988018889018801AA00AA0140
:101420008800811F9F1E8000880080001F7F9F0012
:101430008001070F3FBE3C00183FBF3F070707076B
:1014400048D890D85888509888100000F8F8F87854
:101450007878F8F8F0C0000000C0E0F0F87838388C
:1014600078F8F8F0C000080000F8FCFC1C3C3C7C5C
:1014700035AB17AA950AB7150200F0FFFF1F000051
:1014800000C0F8FF7F0700E0FEFFFF03000080C000
:10149000E0F87F3F070000E0FFFFDFC0C0E0F0F8AA
:1014A00001020102030100003C3F3F3F3C1C1E1EA5
:1014B0000F070301000000000707070707070703DE
:1014C000010100000000000303010101010100000F
:1014D000000000000000000000000000000000000C
:1014E00000000000000080808080C0C0C0E0E0E01C
:1014F000E0E0E0C0E0E0E0C0A0E040E0A0E0C060EC
:1015000000000000000000000080C0E0F0F0D8F80B
:10151000ECECF6F6F3FBF9EDF57FBF413D05050573
:1015200005050505050405050505AD0005050405CA
:101530000000C02010080C0E0F0F0F070707070749
:1015400003030101000000000000FF0000F8046236
:1015500092929292620478000000AA000000005566
:10156000FC0300000000000000404040404060607C
:1015700000000000000000000000FF0000FF00006D
:10158000000000000000FF008040AA70301888D0E2
:101590000304080810101090D0F0F0F0F0F0F0F014
:1015A000F0F0F0F0F0FCFCFCF0F0FF60C0DFDEDFFC
:1015B000DF5F57FF6F5EDD47F3D97C6CD62B949BC2
:1015C00000000000000607070707070707070707CF
:1015D00007070707070707070705060707070301A8
:1015E000000000030408090B0B08080402010203B1
:1015F0000408020110408040102040804080080212
:101600000401804020100201108010204040200082
:10161000000000250028002B002E003100040404E7
:101620000404030405020202020403020202020689
:101630000606060606040402020204040301000072
:101640000000003E5B4F5B3E3E6B4F6B3E1C3E7CA2
:101650003E1C183C7E3C181C577D571C1C5E7F5E50
:101660001C00183C1800FFE7C3E7FF00182418000F
:10167000FFE7DBE7FF30483A060E262979292640A6
:101680007F050507407F05253F5A3CE73C5A7F3ED2
:101690001C1C08081C1C3E7F14227F22145F5F0064
:1016A0005F5F06097F017F006689956A6060606000
:1016B0006094A2FFA29408047E040810207E2010EB
:1016C00008082A1C08081C2A08081E101010100CF4
:1016D0001E0C1E0C30383E3830060E3E0E06000042
:1016E00000000000005F00000007000700147F14E6
:1016F0007F14242A7F2A1223130864623649562055
:10170000500008070300001C2241000041221C0079
:101710002A1C7F1C2A08083E080800807030000838
:1017200008080808000060600020100804023E510C
:1017300049453E00427F400072494949462141499E
:101740004D331814127F1027454545393C4A494905
:101750003141211109073649494936464949291E6F
:10176000000014000000403400000008142241145E
:1017700014141414004122140802015909063E41B0
:101780005D594E7C1211127C7F494949363E4141D8
:1017900041227F4141413E7F494949417F09090931
:1017A000013E414151737F0808087F00417F41009D
:1017B0002040413F017F081422417F404040407F4C
:1017C000021C027F7F0408107F3E4141413E7F0999
:1017D0000909063E4151215E7F09192946264949DA
:1017E000493203017F01033F4040403F1F2040201A
:1017F0001F3F4038403F6314081463030478040318
:101800006159494D43007F414141020408102000C5
:101810004141417F04020102044040404040000336
:1018200007080020545478407F2844443838444402
:101830004428384444287F385454541800087E09FA
:101840000218A4A49C787F0804047800447D40001A
:101850002040403D007F1028440000417F40007C34
:10186000047804787C080404783844444438FC182C
:1018700024241818242418FC7C0804040848545410
:10188000542404043F44243C4040207C1C2040203D
:101890001C3C4030403C44281028444C9090907CA4
:1018A0004464544C440008364100000077000000B6
:1018B0004136080002010204023C2623263C1EA1F8
:1018C000A161123A4040207A385454555921555557
:1018D0007941215454784121555478402054557908
:1018E000400C1E5272123955555559395454545999
:1018F00039555454580000457C410002457D420052
:1019000001457C40F0292429F0F0282528F07C545A
:101910005545002054547C547C0A097F493249497A
:1019200049323248484832324A4848303A414121E7
:101930007A3A42402078009DA0A07D394444443941
:101940003D4040403D3C24FF2424487E4943662BD3
:101950002FFC2F2BFF0929F620C0887E0903205475
:101960005479410000447D413048484A3238404073
:10197000227A007A0A0A727D0D19317D2629292FD3
:1019800028262929292630484D40203808080808EB
:1019900008080808382F10C8ACBA2F102834FA00ED
:1019A000007B000008142A142222142A140895002F
:1019B000220095AA005500AAAA55AA55AA0000001F
:1019C000FF00101010FF00141414FF001010FF008F
:1019D000FF1010F010F0141414FC001414F700FFA2
:1019E0000000FF00FF1414F404FC141417101F105F
:1019F000101F101F1414141F00101010F00000000E
:101A0000001F101010101F10101010F01000000018
:101A1000FF101010101010101010FF10000000FF29
:101A2000140000FF00FF00001F10170000FC04F46A
:101A300014141710171414F404F40000FF00F71422
:101A4000141414141414F700F714141417141010A9
:101A50001F101F141414F4141010F010F000001FC5
:101A6000101F0000001F14000000FC140000F01004
:101A7000F01010FF10FF141414FF141010101F00AA
:101A8000000000F010FFFFFFFFFFF0F0F0F0F0FFAC
:101A9000FFFF0000000000FFFF0F0F0F0F0F384483
:101AA0004438447C2A2A3E147E02020606027E0244
:101AB0007E0263554941633844443C04407E201E05
:101AC0002006027E020299A5E7A5991C2A492A1C34
:101AD0004C7201724C304A4D4D303048784830BC21
:101AE000625A463D3E494949007E0101017E2A2A4B
:101AF0002A2A2A44445F444440514A444040444ACC
:101B000051400000FF0103E080FF000008086B6BFC
:101B1000083612362436060F090F06000018180082
:101B200000001010003040FF0101001F01011E00E5
:101B3000191D1712003C3C3C3C000000000006014F
:101B40001501260137014A015D01720188019F01DB
:101B5000B801D201EE010B022A024B026E0293027F
:101B6000BA02E40210033F037003A403DC0317046A
:101B700055049704DD0427057505C80520067D0674
:101B8000E0064907B8072D08A9082D09B9094D0A2B
:101B9000EA0A900B400CFA0CC00D910E6F0F5A1010
:101BA00053115B1272139A14D41520178018F5196B
:101BB000801B231DDE1EB420A622B524E426342972
:101BC000A72B402E0031EA330037453ABC3D68412F
:101BD0004C456B49C84D68524F57805C00621011EC
:101BE0001213151617181A1C1D1F21232527292C1F
:101BF0002E3134373A3E4145494E52575C62686E49
:101C0000757B838B939CA5AFB9C4D0DCE9F700004A
:101C1000000200090F0000030401000C0000000096
:101C200000000000000000000000000000080B00A1
:101C30000202020100090400000102020000052462
:101C400000100105240101010424020605240600F8
:101C5000010705810310004009040100020A000089
:101C6000000705020240000007058302400000044F
:101C700003090441726475696E6F204C4C43004146
:101C8000726475696E6F204C656F6E6172646F006F
:101C900012010002000000404123368000010102D1
:101CA000030112010002EF020140412336800001CE
:101CB00001020301782311241FBECFEFDAE0DEBF5B
:101CC000CDBF26E0AAE8B1E001C01D92A136B2075F
:101CD000E1F711E0A0E0B1E0EAE1FFE402C0059025
:101CE0000D92AA38B107D9F71EE0CBE5DEE004C0BB
:101CF0002197FE010E94BF23CA35D107C9F70E9470
:101D0000901B0C948B270C940000FC018091C10166
:101D1000811103C08FEF9FEF08959FB7F89482E081
:101D20008093E9002091F20030E01216130614F4BB
:101D300021E030E02115310559F0289884E68093A0
:101D4000C0018091F10080838091F200882319F016
:101D50009FBFC90108958BE68093E800F9CFCF9328
:101D6000DF931F92CDB7DEB76983DC01ED91FC9163
:101D70000280F381E02D41E050E0BE016F5F7F4FB4
:101D800009950F90DF91CF91089583E08093E9004A
:101D90008091F200882319F08AE38093E800089587
:101DA000CF93DF931F92CDB7DEB7FC018485958575
:101DB00097FD05C02FEF3FEF358724870BC0CE017D
:101DC00001960E94850E019719F4898190E002C066
:101DD0008FEF9FEF0F90DF91CF9108950F931F9397
:101DE000CF93DF931F92CDB7DEB78C01FC018485C2
:101DF000958597FF0EC0CE0101960E94850E019732
:101E000019F4298130E002C02FEF3FEFF801358748
:101E10002487F801848595850F90DF91CF911F91DC
:101E20000F910895009769F0FC0101900020E9F7F7
:101E30003197AF01481B590BBC018BEC91E00C941E
:101E40007A1280E090E008958F929F92AF92BF92B5
:101E5000CF92DF92EF92FF920F931F93CF93DF9376
:101E60005C016B018A0180910E01882309F45EC038
:101E70008091C101882309F459C08091BF0180FF7E
:101E800005C08091E00082608093E000E8018AEF65
:101E9000F82E93E0E92E2FE3822E3AE3932E20973B
:101EA00009F43DC08FB7F894E092E9009091E80002
:101EB00095FF06C09091F200282D291B922F01C09A
:101EC00090E08FBF91110AC0FA94FF2079F161E090
:101ED00070E080E090E00E940314E1CF292F30E011
:101EE000C217D3070CF49C2F8FB7F894E092E90047
:101EF0002091E80025FF11C0292F30E0C21BD30B31
:101F0000F601915020F041914093F100FACFC20EBA
:101F1000D31E9091E80095FF13C08FBFC0CF5D988E
:101F200084E68093BE011016110644F081E090E033
:101F3000F5019383828380E090E005C0C80103C06F
:101F40009092E800EACFDF91CF911F910F91FF901F
:101F5000EF90DF90CF90BF90AF909F908F900895BB
:101F6000CF93DF931F92CDB7DEB76091C90180EAAE
:101F700091E069830E94DB266981681721F080EA7D
:101F800091E00E94E3266091CA0181EA91E06983B1
:101F90000E94DB266981681721F081EA91E00E94A6
:101FA000E32689EC91E00F90DF91CF910895CF93D4
:101FB000DF939091C801923009F46EC0C82F292F89
:101FC00030E0F901E45CF94ED491F901EF50FA4F99
:101FD00080839F5F9093C80161E00E942F13D130EE
:101FE00019F0D33039F158C010928000109281005E
:101FF0008091810088608093810080918100816060
:10200000809381008C2F90E0FC01E35EF94EE49117
:10201000F0E0EE0FFF1FE15FF94E25913491309310
:10202000C7012093C601FC01E051FA4E84918093D0
:10203000C50132C0109290001092910080919100E1
:1020400088608093910080919100816080939100DD
:102050008C2F90E0FC01E35EF94EE491F0E0EE0F8E
:10206000FF1FE15FF94E259134913093C401209315
:10207000C301FC01E051FA4E84918093C20180912A
:10208000C801882321F06CE380E00E94B41480E052
:10209000DF91CF910C949F15DF91CF9108952F92EE
:1020A0003F924F925F926F927F928F929F92AF92E8
:1020B000BF92CF92DF92EF92FF920F931F93CF9335
:1020C000DF93CDB7DEB728970FB6F894DEBF0FBE0B
:1020D000CDBF222E312C9C01220D331D37FD30C186
:1020E000803891050CF02CC19B01200F311D37FD6C
:1020F00027C1603471050CF023C1DB0177FF04C0F8
:10210000AA27BB27A61BB70BA770BB279B0177FF8E
:1021100002C0295F3F4F13E0359527951A95E1F7E7
:1021200077FF08C02150310968E070E05B01AA1A0E
:10213000BB0AD501E02FE695E695E695CE2ED12C8B
:10214000077019F00FEFC01AD00AB9017695762FF3
:10215000662777956795680F791F5601A20EB31E03
:10216000BC82AB82412C512CF8E0CF2ED12C8601C1
:102170000A1B1B0B1A830983AB80BC802A153B0505
:1021800009F4DEC02830310509F4DAC02F3F1FEF13
:1021900031070CF4CAC03B01E0E86E0E711C8B01E4
:1021A000015A1D4F1E830D834C0100E010E0021503
:1021B00013050CF0BAC0E0E88E16910409F4B5C01E
:1021C00097FCA8C02F3FFFEF3F0709F4B5C0F80107
:1021D000E40DF51DCD80DE80C618D708AA24A3948F
:1021E000E40FF51FEA1013C0E491C60ED71EF0E00D
:1021F0005F010A2E02C0AA0CBB1C0A94E2F7B88643
:10220000AF82F601B080EF81F885EB292BC0E11099
:1022100017C0E491C60ED71EF0E00A2E02C0EE0FE2
:10222000FF1F0A94E2F75F01A094B094B886AF82D2
:10223000F601A080B12CEF81F885AE22BF2213C039
:10224000E491C60ED71EF0E05F010A2E02C0AA0C70
:10225000BB1C0A94E2F7B886AF82F601B080EF812A
:10226000F885EB255F01F601A082109709F452C0B2
:102270002730310509F44EC0F801E40DF51DAA24FC
:10228000A394EA1011C0E40FF51FE491CE2ED12CD7
:102290005601098002C0B594A7940A94E2F7ED8133
:1022A000FE81D080AD2835C0CD80DE80C618D7082D
:1022B000E40FF51FE11018C0E491C60CD71CAE2E38
:1022C000B12C098002C0B594A7940A94E2F7F501F5
:1022D000E095F095F887EF83F601A080B12CEF81AF
:1022E000F885AE22BF2214C0E491C60CD71CAE2ED6
:1022F000B12CF501098002C0F595E7950A94E2F743
:10230000F887EF83F601B080EF81F885EB255F0158
:10231000F601A0820F5F1F4FED81FE813196FE8393
:10232000ED83FFEF8F1A9F0A42CF2F5F3F4F420C82
:10233000531C60587F4F20CF109709F09DCFEACFF4
:1023400028960FB6F894DEBF0FBECDBFDF91CF91B8
:102350001F910F91FF90EF90DF90CF90BF90AF90C3
:102360009F908F907F906F905F904F903F902F90B5
:10237000089520E08FED91E0B22FB111BFEFFC0185
:102380000024B193B193B193B1930394D1F708951D
:102390000C94120F8F929F92AF92BF92CF92DF92C6
:1023A000EF92FF920F931F93CF93DF93CDB7DEB7DA
:1023B000A1970FB6F894DEBF0FBECDBF6C01990F89
:1023C000EE08FF08F7FE31C0E091CB01F091CC019F
:1023D0000190F081E02D6DE28BEC91E009958C018C
:1023E00022273327A9012C193D094E095F0919A29B
:1023F000CE0181967C019AE0892E912CA12CB12CE2
:10240000CA01B901A50194010E942327605DF7016B
:1024100062937F01211531054105510589F7CF01EF
:102420000E94120F800F911F1DC0A701960119A2D3
:102430008E010F5D1F4F8AE0C82ED12CE12CF12CAC
:10244000CA01B901A70196010E942327605DF80126
:1024500062938F01211531054105510589F7CF019F
:102460000E94120FA1960FB6F894DEBF0FBECDBF2B
:10247000DF91CF911F910F91FF90EF90DF90CF9060
:10248000BF90AF909F908F9008950F931F93CF931D
:10249000DF938C01C0E0D0E0F801EC0FFD1F6491E8
:1024A000662371F0E091CB01F091CC010190F081B5
:1024B000E02D8BEC91E00995892B11F02196ECCF62
:1024C000CE01DF91CF911F910F9108958091E90581
:1024D00081110DC082E08093E50584E08093E605DC
:1024E0001092E8051092E70581E08093E90585EEFA
:1024F00095E00895CF92DF92EF92FF920F931F9392
:10250000CF93DF936C017A018B01C0E0D0E0CE1550
:10251000DF0589F0D8016D918D01D601ED91FC9117
:102520000190F081E02DC6010995892B11F47E01FF
:1025300002C02196ECCFC701DF91CF911F910F917F
:10254000FF90EF90DF90CF9008953FB7F89480917F
:10255000560690915706A0915806B091590626B597
:10256000A89B05C02F3F19F00196A11DB11D3FBFCB
:10257000BA2FA92F982F8827820F911DA11DB11D59
:10258000BC01CD0142E0660F771F881F991F4A9555
:10259000D1F708950E94D923362F90E0FC01E25F25
:1025A000F34E4491FC01E051FA4E2491FC01E35EAC
:1025B000F94E8491882309F451C04423E1F150E09D
:1025C000FA013197EF30F105B0F5EA5AFF4F0C945C
:1025D000BF23909180009F7707C0909180009F7DDE
:1025E00003C090918000977F9093800024C094B5A1
:1025F0009F7702C094B59F7D94BD1DC090919000BF
:102600009F7707C0909190009F7D03C090919000AC
:10261000977F909390000FC09091C0009F7703C068
:102620009091C0009F7D9093C00005C09091C20022
:10263000977F9093C200E82FF0E0EE0FFF1FE15F5D
:10264000F94EA591B4918FB7F894EC91311103C074
:1026500020952E2301C02E2B2C938FBF0895CF934E
:10266000DF9390E0FC01E051FA4E2491FC01E35E1F
:10267000F94E8491882361F190E0880F991FFC0145
:10268000E856FE4FC591D491FC01E15FF94EA5914A
:10269000B491611109C09FB7F89488812095822375
:1026A0008883EC912E230BC0623061F49FB7F894BD
:1026B0003881822F809583238883EC912E2B2C9355
:1026C0009FBF06C08FB7F894E8812E2B28838FBF59
:1026D000DF91CF9108951F93CF93DF93182FEB01D4
:1026E00061E00E942F13209711F460E004C0CF3FF7
:1026F000D10539F461E0812FDF91CF911F910C94C6
:10270000CC12E12FF0E0E25FF34EE4914E2F50E067
:10271000FA013197EF30F10508F06CC0EB59FF4F2B
:102720000C94BF2384B5806884BDC7BD68C084B5E0
:10273000806284BDC8BD63C0809180008068809342
:102740008000D0938900C093880059C08091800098
:10275000806280938000D0938B00C0938A004FC02A
:1027600080918000886080938000D0938D00C0931A
:102770008C0045C080919000806880939000D09339
:102780009900C09398003BC0809190008062809334
:102790009000D0939B00C0939A0031C0809190002C
:1027A000886080939000D0939D00C0939C0027C0C8
:1027B0008091C00080688093C0008091C0008F7BB2
:1027C0008093C000C093CF001AC08091C000806287
:1027D0008093C000C093D00012C08091C200886076
:1027E0008093C2008091C2008B7F8093C200C0930F
:1027F000D20005C0C038D1050CF07CCF76CFDF9178
:10280000CF911F9108958F929F92AF92BF92CF92D6
:10281000DF92EF92FF926B017C010E94A5124B01A7
:102820005C01C114D104E104F104F1F00E94A5128D
:10283000DC01CB0188199909AA09BB09883E93409C
:10284000A105B10570F321E0C21AD108E108F10831
:1028500088EE880E83E0981EA11CB11CC114D1041F
:10286000E104F10419F7DDCFFF90EF90DF90CF90F6
:10287000BF90AF909F908F9008951F920F920FB6C8
:102880000F9211242F933F938F939F93AF93BF93F6
:102890008091520690915306A0915406B09155062E
:1028A0003091510623E0230F2D3720F40196A11D0E
:1028B000B11D05C026E8230F0296A11DB11D20936E
:1028C00051068093520690935306A0935406B093FA
:1028D00055068091560690915706A0915806B091E2
:1028E00059060196A11DB11D809356069093570677
:1028F000A0935806B0935906BF91AF919F918F91C5
:102900003F912F910F900FBE0F901F9018958FB190
:102910002CB193B130E02095309520743327A90174
:1029200023E0559547952A95E1F7292F30E020952A
:102930003095207133273595279535952795242B8C
:102940008095807F822B0895FC0121912EBD9C5F94
:1029500021910DB407FEFDCF2EBDE817F907C1F791
:102960000DB407FEFDCF0895CF92DF92EF92FF9254
:102970000F931F93CF93E82FF0E0E45CF94EC491DE
:10298000E62FF0E0603330F4E252F44EE4910E2F83
:1029900010E006C0EE0FFF1FE252F54E05911491B4
:1029A0006801E12CF12C60E074E284EF90E0A70173
:1029B00096010E94F126BA01A9014150510961090D
:1029C00071094115510581E06807710580F060E9E2
:1029D00070ED83E090E0A70196010E94F126BA0114
:1029E000A901415051096109710983E001C081E0E9
:1029F000C130C9F0C33031F590919100987F892B97
:102A00008093910050939900409398001093500642
:102A100000934F0681E080934E06809171008260A2
:102A2000809371000FC090918100987F892B8093D3
:102A30008100509389004093880080916F008260EC
:102A400080936F00CF911F910F91FF90EF90DF90D7
:102A5000CF9008951F920F920FB60F9211242F93CB
:102A60003F938F939F93AF93BF93EF93FF93809187
:102A70004706882309F44DC080914306909144068F
:102A8000A0914506B0914606892B8A2B8B2B51F1DC
:102A90008091C501E091C601F091C701908189271D
:102AA00080838091430690914406A0914506B091A1
:102AB0004606181619061A061B06A4F58091430649
:102AC00090914406A0914506B09146060197A10950
:102AD000B1098093430690934406A0934506B093B2
:102AE000460620C01092470680916F008D7F80932C
:102AF0006F009091C501E091C601F091C7018081FE
:102B0000282F30E0892F90E08095909582239323A1
:102B100008C08091C501E091C601F091C701908184
:102B200089278083FF91EF91BF91AF919F918F9102
:102B30003F912F910F900FBE0F901F901895E82F87
:102B4000F0E0E45CF94EE491E13019F0E33069F033
:102B5000089580916F008D7F80936F009091C501E3
:102B6000E091C601F091C70108C010924E06909105
:102B7000C201E091C301F091C4018081282F30E0AF
:102B8000892F90E0809590958223932380830895E8
:102B90001F920F920FB60F9211242F933F934F93D2
:102BA0005F936F937F938F939F93AF93BF93EF93B5
:102BB000FF9380914E06882349F08091C201E091F5
:102BC000C301F091C40190818927808380918A019B
:102BD000882309F493C080914A0690914B06A091F6
:102BE0004C06B0914D06892B8A2B8B2B09F486C09D
:102BF00080914A0690914B06A0914C06B0914D06EB
:102C00000197A109B10980934A0690934B06A093BE
:102C10004C06B0934D06892B8A2B8B2B09F06EC086
:102C2000E0914806F0914906BF016F5F7F4F7093B6
:102C30004906609348064491942F907F842F8F70AB
:102C4000903819F40E949F15EBCF903981F4329699
:102C5000F0934906E0934806FB0164919091C80106
:102C60008917F0F667FDDCCF0E94B414D9CF903EEF
:102C700029F41092490610924806D2CF903F19F4D9
:102C800010928A013BC097FDCBCF3296F093490654
:102C9000E0934806FB01249130E0342BA0914F06CD
:102CA000B09150060E9445276C507E4F8F4F9F4F2A
:102CB00028EE33E040E050E00E94232720934A06AC
:102CC00030934B0640934C0650934D0680914A0634
:102CD00090914B06A0914C06B0914D06892B8A2B02
:102CE0008B2B61F481E090E0A0E0B0E080934A0695
:102CF00090934B06A0934C06B0934D06FF91EF9135
:102D0000BF91AF919F918F917F916F915F914F9103
:102D10003F912F910F900FBE0F901F901895603824
:102D2000710518F54034510500F5A42FA695A69518
:102D3000A695B0E047705527B695BA2FAA27B79544
:102D4000A7956A0F7B1FFC01E60FF71F81E090E05B
:102D500001C0880F4A95EAF7222319F09489892B3C
:102D600003C0809594898923848B08952F923F9284
:102D70004F925F926F927F928F929F92AF92BF928B
:102D8000CF92DF92EF92FF920F931F93CF93DF9337
:102D9000CDB7DEB72A970FB6F894DEBF0FBECDBF12
:102DA0006A3091F4FC01E85EFB4F4081329720814C
:102DB000318158E0459F200D311D1124318320833E
:102DC000329711821082C1C06D3009F4BEC09A875B
:102DD0008987885E9B4F9C838B83DC012C90E985DF
:102DE000FA85EA5EFB4F60807180E985FA85EC5ECA
:102DF000FB4FFA83E9830081118100381105D4F07B
:102E0000AB81BC812C91422F50E0E981FA81808115
:102E10009181F6E02F9F800D911D1124A981BA8127
:102E20008D939C93E985FA85E75EFB4F2081211104
:102E30005EC08BC0B0E46B16710414F7C801E5E006
:102E40002E9E800D911D112418161906CCF6422CC9
:102E5000512CC301F8E02F9E800D911D11241816EE
:102E6000190674F655E0659F900111243F832E8367
:102E7000E12CF12C85E0E816F10441F0EE81FF81B0
:102E8000EE0DFF1DE25CF94E349001C0312C630160
:102E900038E0932D91709D834801882D801B821509
:102EA000B0F456018A2D8C19821568F42D81A50184
:102EB000B40189859A8538870E948F16AFEFAA1AC8
:102EC000BA0A3885EFCFBFEF8B1A9B0AE6CF36944C
:102ED0003150C40CD51C3111DCCFEFEFEE1AFE0AD5
:102EE000040D151DF6E0EF16F10421F689CF6AEF07
:102EF00064039001659F300D112420583F4F28171F
:102F000039071CF5A985BA85ED91FC9111970190BF
:102F1000F081E02D6AE0CD012A960FB6F894DEBF6D
:102F20000FBECDBFDF91CF911F910F91FF90EF901A
:102F3000DF90CF90BF90AF909F908F907F906F90D9
:102F40005F904F903F902F9009942A960FB6F89477
:102F5000DEBF0FBECDBFDF91CF911F910F91FF90CC
:102F6000EF90DF90CF90BF90AF909F908F907F9029
:102F70006F905F904F903F902F9008951092920124
:102F80001092910180E890E09093010180930001FC
:102F900081E090E090938C0180938B0110929401DA
:102FA0001092930110928E0110928D011092900157
:102FB00010928F01109296011092950184E190E099
:102FC000909305018093040181E080930201809336
:102FD00003010E94CB2664EF71E00E94AB23845D65
:102FE0009E4F90939601809395010895FC018485EE
:102FF000958597FD0BC09FB7F89482E08093E90018
:103000008091F2009FBF90E0019608959FB7F894D9
:1030100082E08093E9008091F2009FBF90E00895E4
:1030200040915F065091600620915D0630915E06EA
:1030300042175307B4F49091E8009570E1F3909132
:10304000E80092FD19C08093F10080915F06909195
:10305000600601968F739927892B19F48EEF809360
:10306000E80080915F06909160060196909360065B
:1030700080935F0681E0089580E00895CF92DF920B
:10308000EF92FF920F931F93CF93DF931F92CDB7D1
:10309000DEB7182F062FE42E862F880F8E5F9983B8
:1030A0000E94101883E00E941018F12EC12E998101
:1030B000D92E8C2D8F19801798F4F601E7FE02C0E7
:1030C000849101C080810E941018182F80E00E9416
:1030D00010188123FFEFCF1ADF0A8111EACF01C058
:1030E00081E00F90DF91CF911F910F91FF90EF90B2
:1030F000DF90CF900895DF92EF92FF920F931F938E
:10310000CF93DF93D82E8A017B01E40EF51EEB01ED
:10311000CE15DF0571F0D7FE03C0FE01849101C01A
:1031200088810E94101821968111F2CF8FEF9FEFB6
:1031300001C0C801DF91CF911F910F91FF90EF90D7
:10314000DF900895615030F02091F100FC01208360
:103150000196F8CF289884E68093C00108950F93D4
:103160001F93CF93DF931F92CDB7DEB782E08983A1
:1031700042E450E06DE27CE180E80E947B180E940E
:103180006612DC0112960D911C9113970115110521
:1031900069F0D801ED91FC910280F381E02DBE0130
:1031A0006F5F7F4FC801099597FF07C089810F9016
:1031B000DF91CF911F910F910895F801008511853E
:1031C000E5CF1F920F920FB60F9211248F939F930A
:1031D0008091E1009091E100937F9093E10083FF63
:1031E0000FC01092E90091E09093EB001092EC0078
:1031F00092E39093ED001092C10198E09093F0005B
:1032000082FF20C093E09093E9009091F20099230F
:1032100019F09AE39093E8009091BE01992339F058
:103220009091BE0191509093BE01992389F19091A4
:10323000C001992339F09091C00191509093C00141
:10324000992341F184FF10C08091E2008E7E81605D
:103250008093E2008091E1008F7E8093E100809175
:10326000BF018E7E806111C080FF16C08091E20098
:103270008E7E80618093E2008091E1008E7E80935B
:10328000E1008091BF018E7E81608093BF0104C008
:103290005D9ACDCF289AD6CF9F918F910F900FBE78
:1032A0000F901F9018951F920F920FB60F92112436
:1032B000CF92DF92EF92FF920F931F932F933F9342
:1032C0004F935F936F937F938F939F93AF93BF932E
:1032D000EF93FF93CF93DF93CDB7DEB76C97DEBF4D
:1032E000CDBF1092E9008091E80083FFFAC168E049
:1032F000CE0145960E94A21882EF8093E8008D8946
:1033000087FF05C09091E80090FFFCCF03C09EEFBF
:103310009093E800982F907609F0C6C09E892F8977
:10332000188D91110CC0803829F480915B06809330
:10333000F10002C01092F1001092F10047C1422F3B
:1033400050E0512B913051F4811140C14130510571
:1033500009F03CC180915B068D7F0BC0933061F416
:10336000811134C14130510509F030C180915B06B3
:10337000826080935B062AC1953041F48091E80019
:1033800080FFFCCF20682093E30020C1963009F035
:103390005FC0EB8CFC8C1092E900109260061092DA
:1033A0005F06123091F510925E0610925D060E9443
:1033B000AF1899E0BE016F5F7F4FDB01E92F1D92CF
:1033C000EA95E9F799831A8391E09E8390EA9887BA
:1033D0009AEF998720915F0630916006275F3F4FF3
:1033E0003C832B838D831092E9001092600610922B
:1033F0005F06F0925E06E0925D0649E050E080E0F4
:103400000E947B180E94AF18E1C0F0925E06E09225
:103410005D060E946612DC011296ED90FC901397F7
:10342000E114F10409F4C0C0D701ED91FC910480CE
:10343000F581E02DBE016B5E7F4FC70109950097B6
:1034400019F00CF0C3C0C6C0F701E084F184E8CFE6
:10345000973009F4BFC0983021F481E08093F100E7
:10346000B5C0993009F0B2C0837009F0B3C0E4E38D
:10347000F1E081E021E036E39081992361F08093CF
:10348000E9002093EB0091919093EC003093ED00D4
:103490008F5F873089F78EE78093EA001092EA0009
:1034A0008F898093C10192C08B8D9C8D1092E90011
:1034B0001092600610925F0690935E0680935D0600
:1034C000898D811156C08E899D89913A59F4813236
:1034D00009F080C047E050E067E071E080E00E94C2
:1034E0007B1874C0913209F075C0833289F4888DDD
:1034F00090E0982F88272F89822BA0E0B0E080935E
:103500000F0190931001A0931101B09312015EC0BE
:10351000803269F48091E80082FFFCCF67E087E0A9
:1035200091E00E94A2188BEF8093E80006C08232DF
:1035300009F04CC08F8980930E0180915A06882330
:1035400019F0EEEFFAE002C0E0E0F8E08091070148
:1035500090910801A0910901B0910A01803B94402B
:10356000A105B10509F088C080910E0180FFA0C0BF
:1035700083C00E946612DC0112960D911C91139774
:103580000115110539F1D801ED91FC910190F081FF
:10359000E02DBE016B5E7F4FC8010995811116C0F9
:1035A000F80100851185ECCF1130C1F0133091F492
:1035B0008F89882309F455C08230E9F440E860E13E
:1035C0008FE79CE10E943E18882321F08EEF8093C4
:1035D000E80087C081E28093EB0083C08B8D9C8DD7
:1035E000089711F410935C0680915C06811136C037
:1035F00060E97CE138C0813029F440E86BE083E782
:103600009CE1E0CF833031F70E946612DC01129614
:10361000ED90FC9013978E010F5F1F4F6801E1142E
:10362000F10479F0D701ED91FC910680F781E02D4E
:10363000B801C7010995080F111DF701E084F18455
:10364000EECFD8011C92F60101900020E9F73197E6
:10365000BF016C197D0940E0C601B4CF62EA7CE18C
:1036600002C06FE67CE16115710509F4B3CFFB017F
:10367000449150E080E833CF0FB6F894A89580913C
:103680006000886180936000109260000FBEA89572
:10369000EE3F2AE0F20739F08091FE0A9091FF0A8E
:1036A0009183808393CF1092FF0A1092FE0A8ECFEF
:1036B000EE3F8AE0F80731F0808191819093FF0A14
:1036C0008093FE0A87E797E7918380839BE088E1F8
:1036D0000FB6F894A895809360000FBE9093600099
:1036E00075CF6C960FB6F894DEBF0FBECDBFDF91DD
:1036F000CF91FF91EF91BF91AF919F918F917F916A
:103700006F915F914F913F912F911F910F91FF907A
:10371000EF90DF90CF900F900FBE0F901F901895F5
:10372000CF93DF931F92CDB7DEB7789484B58260D4
:1037300084BD84B5816084BD85B5826085BD85B555
:10374000816085BD80916E00816080936E001092D3
:10375000810080918100826080938100809181004E
:1037600081608093810080918000816080938000DF
:10377000809191008260809391008091910081609E
:10378000809391008091900081608093900080915F
:10379000C10084608093C1008091C10082608093E9
:1037A000C1008091C10081608093C1008091C300FD
:1037B00081608093C3008091C00082608093C000CC
:1037C0008091C20081608093C20080917A00846001
:1037D00080937A0080917A00826080937A00809151
:1037E0007A00816080937A0080917A00806880936B
:1037F0007A001092C10110925B061092BF01809175
:10380000D70081608093D70080EA8093D80089B583
:10381000806189BD89B5826089BD09B400FEFDCF94
:1038200061E070E080E090E00E9403148091D80095
:103830008F7C80618093D8008091E000807F8093AE
:10384000E0008091E1008E7E8093E1008DE0809326
:10385000E200559A209AEEEFFFE7859194918B3F15
:103860009C4D19F481E080935A061FB7F89480911B
:103870009801811127C0EEE2F6E18491E1E0F6E1E2
:103880009491E82FF0E0EE0FFF1FE856FE4FA59150
:10389000B491EC91E92321F461E081E10E94CC1222
:1038A00061E081E10E942F138CB580618CBD8CB5E5
:1038B00080648CBD61E08FE00E942F1361E080E1A5
:1038C0000E942F13809198018F5F809398011FBFF2
:1038D00003EB11E0F80184910E5F1F4F3196649164
:1038E000882319F00E942F13F5CF61E086E00E9433
:1038F000CC1261E070E080E090E00E94031460E090
:1039000086E00E94CC126AE070E080E090E00E94C5
:10391000031461E086E00E94CC12E9E2F6E1E49152
:10392000F0E0EE0FFF1FE15FF94E859194919093C7
:103930009E0180939D01ECEFF5E1E491E0939C0101
:10394000E1E2F6E1E491F0E0EE0FFF1FE15FF94EF6
:103950008591949190939B0180939A01E4EFF5E116
:10396000E491E09399018CB58C7F8CBD8DB581601D
:103970008DBDE0919D01F0919E01908180919C010F
:10398000982B9083A0919A01B0919B012C919091DA
:103990009901909592239C939081809589238083AF
:1039A000E6EAF1E021E0E33BF20749F084918EBDC5
:1039B00000000DB407FEFDCF8EB53196F3CFE09138
:1039C0009A01F0919B01908180919901892B8083CC
:1039D000E0919D01F0919E01908180919C018095E4
:1039E000892380838091640081608093640080914A
:1039F000640082608093640080916400806880939A
:103A0000640080916400806480936400809165000C
:103A10008160809365000E94871487FF1AC080E050
:103A200094E01EBC00000DB407FEFDCF2EB501973B
:103A3000C1F760E070E08AE00E946B1360E070E024
:103A40008BE00E946B1360E070E089E00E946B13D2
:103A5000FFCF4EEEA42EBB24BA9418E1CC24CA9416
:103A6000D12C812F8A19B601681B71098AE00E9446
:103A70006B136FEF70E08BE00E946B136FEF70E0E1
:103A800089E00E946B130E94B911EE24E39400E1D7
:103A900028E548EE50E0B50184E190E00E944F1027
:103AA0008FED91E00E94A4146BE170E080E090E063
:103AB0000E94031430EFA31206C06AEF70E080E0AA
:103AC00090E00E9403148FEFA81AB80A99E1A91692
:103AD000B10439F66EEE72E080E090E00E940314CB
:103AE0006FEF70E08AE00E946B136FEF70E08BE085
:103AF0000E946B136FEF70E089E00E946B1385E00A
:103B00000E94D70F8DE00E94D70F10928A0182E0A9
:103B100090E00E94DB26882369F080916400877F13
:103B20008093640080916500877F8093650081E0C9
:103B30008093970186E98093D10186E08093D40138
:103B40008FED91E00E94A41480E090E00E94D026C6
:103B500080EA91E00E94DB268093C90181EA91E02E
:103B60000E94DB268093CA0194E1692E712C2EE11C
:103B7000A22EB12C38E2432E512C82E0282E312C7B
:103B80000E94B9118091BC019091BD0182309105D4
:103B900009F4CAC034F4009781F0019709F455C0C4
:103BA0004DC58F30910509F471C08031910509F43C
:103BB0009AC0039709F042C50FC4EE24E39400E3D2
:103BC00020E340ED54E160E070E080E090E00E948E
:103BD0004F1020E340EB53E160E070E080E390E0C1
:103BE0000E944F1020E340E952E160E070E080E67F
:103BF00090E00E944F10B092E005A092DF058FE2A6
:103C000090E09093E2058093E1058AE391E00E94C1
:103C1000C8117092E0056092DF0587E390E0909311
:103C2000E2058093E10587E491E00E94C8110E94BB
:103C3000871483FF05C080910601811113C5FEC45E
:103C40000E94871482FDF7CFF9C4EE24E39400E1CB
:103C500020E140E752E163E370E08EE690E00E94ED
:103C60004F101092E0051092DF051092E2051092BD
:103C7000E1058FE092E10E9445120E94871483FFC4
:103C8000DDC4809106018111F6C4D8C4EE24E3940A
:103C900000E120E140E752E163E370E08EE690E06E
:103CA0000E944F101092E0051092DF051092E2057D
:103CB0001092E10589ED91E10E9445120E9487145E
:103CC00082FF08C00E94871487FF04C0809106010C
:103CD0008111D8C40E94871483FFB0C4809106016B
:103CE0008111DFC4ABC4EE24E39400E120E140E79E
:103CF00052E163E370E08EE690E00E944F10109274
:103D0000E0051092DF051092E2051092E10586EAC7
:103D100091E10E9445120E94871483FF8FC4809115
:103D200006018111C3C48AC41092BB0180900401B2
:103D300090900501009195011091960108191909BB
:103D400010939601009395010E94871483FF1CC075
:103D5000809106018823C1F0809103018823A1F09E
:103D600080910201882381F01092060110920301D4
:103D7000013811054CF080919301909194010A97BC
:103D800090939401809393011092BA011092B9011B
:103D9000E090B901F090BA01F0E8EF16F1041CF5DB
:103DA0001092B8011092B701C090B701D090B8013D
:103DB000B6E2CB16D1047CF421E0A601B7018BEC6E
:103DC00091E00E948F16AFEFCA1ADA0AD092B801BA
:103DD000C092B701E9CFEFEFEE1AFE0AF092BA01F6
:103DE000E092B901D5CFC80108978837910598F4BA
:103DF000809102018823B9F080910301882399F012
:103E00008091930190919401880E991E9092940153
:103E10008092930108C0083011052CF480910301B1
:103E200081111092020180910201882309F482C05D
:103E30008091030181117EC0809191019091920146
:103E400003969093920180939101809193019091B8
:103E50009401843691052CF04996909394018093B7
:103E600093018091930190919401009791F020919A
:103E70008F0130919001280F391F309390012093CA
:103E80008F0190938E0180938D0110929401109276
:103E900093010E94871483FF4AC080910601882302
:103EA00009F445C08091000190910101181619068E
:103EB000F4F11092060180918B0190918C01019692
:103EC00090938C0180938B010E94CB266CE271E071
:103ED0000E94AB23825A9E4F909396018093950146
:103EE00000918B0110918C01043111050CF0E7C396
:103EF0000E94CB26065F1F4F6EE070E00E94AB234E
:103F0000080F191F109305010093040181E08093AD
:103F100003013092BD012092BC01109292011092D7
:103F2000910120E830E0309301012093000181E00D
:103F30008093BB0180910201811132C00E948714DD
:103F400083FF2BC080910601882339F18091000105
:103F5000909101011816190604F110920601A3E0D0
:103F6000B0E0B093BD01A093BC01109292011092F9
:103F7000910180918F01909190012091C901309120
:103F8000CA01281739074CF41816190634F490930F
:103F9000CA018093C9010E94B00F81E08093BB01E8
:103FA000EE24E39404E420E346EE50E166E270E0A0
:103FB00080E090E00E944F1020E346EE50E166E280
:103FC00070E080E390E00E944F1020E346EE50E165
:103FD00066E270E080E690E00E944F10C09095018C
:103FE000D0909601E12C00E320E346EC5FE061E035
:103FF00070E0C6010E944F10EE24E39420E346EAED
:104000005EE061E070E0C6010E944F10460130E3BF
:10401000830E911CE12C20E346E85DE061E070E056
:10402000C4010E944F10EE24E39420E346E65CE0D6
:1040300061E070E0C4010E944F10460180E6880EE6
:10404000911CE12C20E346E45BE061E070E0C401F8
:104050000E944F10EE24E39420E346E25AE061E030
:1040600070E0C4010E944F1046019FE8890E911C28
:10407000E12C20E346E059E061E070E0C4010E94D9
:104080004F10EE24E39420E346EE57E061E070E049
:10409000C4010E944F104601AFEB8A0E911CE12C27
:1040A00020E346EC56E061E070E0C4010E944F104E
:1040B000EE24E39420E346EA55E061E070E0C401B9
:1040C0000E944F104601BFEE8B0E911CE12C20E3A5
:1040D00046E854E061E070E0C4010E944F10EE2415
:1040E000E39420E346E653E061E070E0C4010E94FF
:1040F0004F104601E2EE8E1AEEEF9E0AE12C20E30D
:1041000046E059E061E070E0C4010E944F10EE24E7
:10411000E39420E346EE57E061E070E0C4010E94C2
:104120004F104601F2EB8F1AFEEF9F0AE12C20E3BD
:1041300046EC56E061E070E0C4010E944F10EE24AE
:10414000E39420E346EA55E061E070E0C4010E9498
:104150004F10460122E8821A2EEF920AE12C20E34A
:1041600046E854E061E070E0C4010E944F10EE2484
:10417000E39420E346E653E061E070E0C4010E946E
:104180004F10309102013983332309F44CC08090E1
:1041900091019090920181149104A9F4E12C0AE11B
:1041A0002AE14EEF52E06CE170E085E090E00E9481
:1041B0004F10EE24E3942AE146E952E06CE170E00E
:1041C00085E090E02EC08FE088169104B4F49BE166
:1041D000890E911CE12C0AE12AE14EE252E0B40181
:1041E00087E090E00E944F10EE24E3942AE146EC31
:1041F00051E0B40187E090E014C0E12C0AE12AE12B
:104200004EEF52E06BE270E089E090E00E944F10C8
:10421000EE24E3942AE146E952E06BE270E089E0A3
:1042200090E00E944F108091BB01882309F406C2E0
:1042300080910001909101011816190654F4A2EA28
:10424000CA16AEEFDA062CF408979093010180931A
:1042500000011092B8011092B701E090B701F09000
:10426000B8010091000110910101F0E4EF16F10492
:104270004CF5C8018E0D9F1D9093BA018093B90132
:10428000005C1F4F0E0D1F1DC090B901D090BA01E8
:10429000C016D1067CF420E0A701B6018BEC91E0BA
:1042A0000E948F16BFEFCB1ADB0AD092BA01C092E0
:1042B000B901EACFEFEFEE1AFE0AF092B801E092F0
:1042C000B701CBCF3981332309F444C0045D1F4FBC
:1042D0001093E0050093DF057092E2056092E1051E
:1042E00087E591E00E94C811809100019091010141
:1042F000C7969093E0058093DF05B092E205A09207
:10430000E10580918D0190918E0118161906FCF43B
:10431000853691052CF09F938F93ADE5B1E004C0F5
:104320009F938F93A2E6B1E0BF93AF93AFE9B1E063
:10433000BF93AF930E94DE238FE991E00E94C811E2
:104340000F900F900F900F900F900F9022C00E942F
:10435000CA111FC0035D1F4F1093E0050093DF05D6
:104360007092E2056092E10586E691E00E94C81134
:104370008091000190910101C7969093E005809390
:10438000DF05B092E205A092E1058AE691E00E9485
:10439000C8118091000190910101805C9F4F909322
:1043A000E0058093DF055092E2054092E10580919F
:1043B0008F01909190010E94CA118091000190910B
:1043C0000101EE24E39400E120E140E752E163E3E0
:1043D00070E0805A9F4F30C180919101909192017D
:1043E000803491050CF050C0049690939201809314
:1043F00091011092B8011092B7010091B70110918C
:10440000B8010632110514F51092BA011092B901E3
:10441000E090B901F090BA0120E8E216F1047CF4D2
:1044200021E0A801B7018BEC91E00E948F16FFEF0D
:10443000EF1AFF0AF092BA01E092B901E9CF0F5FDB
:104440001F4F1093B8010093B701D7CFEE24E39428
:1044500004E420E346EE50E166E270E080E090E0A4
:104460000E944F1020E346EE50E166E270E080E3E8
:1044700090E00E944F1020E346EE50E166E270E0CB
:1044800080E690E00E944F101092B8011092B701A0
:104490000091B7011091B801003411052CF510936B
:1044A000BA010093B90168013FE3C30ED11CE0904B
:1044B000B901F090BA01CE14DF047CF020E0A8012D
:1044C000B7018BEC91E00E948F168FEFE81AF80A83
:1044D000F092BA01E092B901EACF0F5F1F4F10933B
:1044E000B8010093B701D4CFC0909101D090920150
:1044F00080E490E08C199D099093B8018093B701F6
:104500000091B7011091B8010034110514F5109213
:10451000BA011092B901E090B901F090BA01A0E897
:10452000EA16F1047CF420E0A801B7018BEC91E0DD
:104530000E948F169FEFE91AF90AF092BA01E092F1
:10454000B901E9CF0F5F1F4F1093B8010093B70176
:10455000D7CF09E210E01093E0050093DF0585E472
:1045600090E08C199D099093E2058093E10580E726
:1045700091E00E94C81120919101309192018FE445
:1045800090E0821B930B1093E0050093DF0590935E
:10459000E2058093E105809190018F9380918F01D6
:1045A0008F938FE791E09F938F93AFE9B1E0BF9333
:1045B000AF930E94DE238FE991E00E94C811209101
:1045C00091013091920188E690E0821B930B29E1E2
:1045D00030E03093E0052093DF059093E20580936F
:1045E000E1058091CA018F938091C9018F938AE779
:1045F00091E09F938F93AFE9B1E0BF93AF930E9497
:10460000DE238FE991E00E94C8110E9487140FB643
:10461000F894DEBF0FBECDBF83FF04C080910601BA
:10462000811159C0EE24E39400E120E140E752E11A
:1046300063E370E08EE690E00E944F1080910601E7
:10464000811104C00E94871483FF4EC08FED91E05A
:104650000E94A41480E090E0892B09F491CA0E9482
:1046600000008BCA81E090E09093BD018093BC0173
:1046700010920601E3CF8FE090E09093BD0180930C
:10468000BC0118C080E190E09093BD018093BC0113
:10469000109206011092CA011092C9010E94B00F37
:1046A00019CB3092BD012092BC0104C01092BD0113
:1046B0001092BC01109206010E94BE17BFCF0E944B
:1046C000CB2664E170E00E94AB234E9690930501E7
:1046D000809304011BCC3092BD012092BC0110924A
:1046E00006010E94BE179ECF81E080930601AECFE7
:1046F000E3EFF5E01382128288EE93E0A0E0B0E0F1
:1047000084839583A683B7838FE191E0918380832F
:104710008FEF9FEF95878487EBECF1E01382128295
:104720008FE291E0918380838CE3868380E18187AF
:104730001086178216861786108A118A128A10929E
:10474000E0051092DF051092E2051092E10581E08C
:104750008093E305089597FB072E16F4009407D085
:1047600077FD09D00E94C52307FC05D03EF4909543
:1047700081959F4F0895709561957F4F0895EE0F35
:10478000FF1F0590F491E02D0994AA1BBB1B51E17A
:1047900007C0AA1FBB1FA617B70710F0A61BB70BB1
:1047A000881F991F5A95A9F780959095BC01CD0156
:1047B000089581E090E0F8940C948B27AEE0B0E08F
:1047C000E4EEF3E20C9462270D891E8986E08C8367
:1047D0001A8309838FEF9FE79E838D83AE01475E27
:1047E0005F4F6F89788DCE0101960E9401242F8141
:1047F0003885F801E20FF31F10822E96E4E00C9446
:104800007E27ACE0B0E0E7E0F4E20C9454277C01B2
:104810006B018A01FC0117821682838181FFBDC171
:10482000CE0101964C01F7019381F60193FD85912C
:1048300093FF81916F01882309F4ABC1853239F46C
:1048400093FD859193FF81916F01853229F4B70122
:1048500090E00E94E925E7CF512C312C20E0203256
:10486000A0F48B3269F030F4803259F0833269F46D
:1048700020612CC08D3239F0803339F4216026C09C
:104880002260246023C0286021C027FD27C030EDAE
:10489000380F3A3078F426FF06C0FAE05F9E300DFC
:1048A0001124532E13C08AE0389E300D1124332E6C
:1048B00020620CC08E3221F426FD6BC1206406C03C
:1048C0008C3611F4206802C0883641F4F60193FD5D
:1048D000859193FF81916F018111C1CF982F9F7DA9
:1048E0009554933028F40C5F1F4FFFE3F9830DC0FC
:1048F000833631F0833771F0833509F05BC022C015
:10490000F801808189830E5F1F4F44244394512C0A
:10491000540115C03801F2E06F0E711CF801A0803F
:10492000B18026FF03C0652D70E002C06FEF7FEFFE
:10493000C5012C870E94DE252C0183012C852F7751
:10494000222E17C03801F2E06F0E711CF801A08012
:10495000B18026FF03C0652D70E002C06FEF7FEFCE
:10496000C5012C870E94D3252C012C852068222E7E
:10497000830123FC1BC0832D90E048165906B0F438
:10498000B70180E290E00E94E9253A94F4CFF50166
:1049900027FC859127FE81915F01B70190E00E947D
:1049A000E92531103A94F1E04F1A510841145104AD
:1049B00071F7E5C0843611F0893639F5F80127FF23
:1049C00007C060817181828193810C5F1F4F08C095
:1049D00060817181072E000C880B990B0E5F1F4FB1
:1049E0002F76722E97FF09C09095809570956195EE
:1049F0007F4F8F4F9F4F2068722E2AE030E0A40136
:104A00000E942126A82EA81844C0853729F42F7E9D
:104A1000B22E2AE030E025C0F22FF97FBF2E8F366C
:104A2000C1F018F4883579F0B4C0803719F08837B0
:104A300021F0AFC02F2F2061B22EB4FE0DC08B2D00
:104A40008460B82E09C024FF0AC09F2F9660B92E3B
:104A500006C028E030E005C020E130E002C020E1DF
:104A600032E0F801B7FE07C06081718182819381D5
:104A70000C5F1F4F06C06081718180E090E00E5F87
:104A80001F4FA4010E942126A82EA818FB2DFF77F6
:104A90007F2E76FE0BC0372D3E7FA51450F474FE9A
:104AA0000AC072FC08C0372D3E7E05C0BA2C372DD7
:104AB00003C0BA2C01C0B52C34FF0DC0FE01EA0DB5
:104AC000F11D8081803311F4397E09C032FF06C0A8
:104AD000B394B39404C0832F867809F0B39433FD64
:104AE00013C030FF06C05A2CB31418F4530C5B18D3
:104AF000B32CB31468F4B70180E290E03C870E94C5
:104B0000E925B3943C85F5CFB31410F43B1801C0EC
:104B1000312C34FF12C0B70180E390E03C870E9443
:104B2000E9253C8532FF17C031FD03C088E790E0DE
:104B300002C088E590E0B7010CC0832F867859F059
:104B400031FF02C08BE201C080E237FD8DE2B70188
:104B500090E00E94E925A51438F4B70180E390E0C5
:104B60000E94E9255A94F7CFAA94F401EA0DF11DA9
:104B70008081B70190E00E94E925A110F5CF332094
:104B800009F451CEB70180E290E00E94E9253A9401
:104B9000F6CFF7018681978102C08FEF9FEF2C96A9
:104BA000E2E10C947027FC01059061507040011007
:104BB000D8F7809590958E0F9F1F0895FC01615046
:104BC000704001900110D8F7809590958E0F9F1F2F
:104BD00008950F931F93CF93DF93FB01238121FD52
:104BE00003C08FEF9FEF28C022FF16C04681578178
:104BF000248135814217530744F4A081B1819D017E
:104C00002F5F3F4F318320838C93268137812F5F25
:104C10003F4F3783268310C0EB01092F182F0084E4
:104C2000F185E02D0995892BE1F68E819F81019612
:104C30009F838E83812F902FDF91CF911F910F91B2
:104C40000895FA01AA27283051F1203181F1E89422
:104C50006F936E7F6E5F7F4F8F4F9F4FAF4FB1E06F
:104C60003ED0B4E03CD0670F781F891F9A1FA11D6A
:104C7000680F791F8A1F911DA11D6A0F711D811D6B
:104C8000911DA11D20D009F468943F912AE0269F30
:104C900011243019305D3193DEF6CF010895462F8F
:104CA0004770405D4193B3E00FD0C9F7F6CF462F70
:104CB0004F70405D4A3318F0495D31FD40524193D9
:104CC00002D0A9F7EACFB4E0A69597958795779596
:104CD0006795BA95C9F700976105710508959B011D
:104CE000AC010A2E06945795479537952795BA95A6
:104CF000C9F7620F731F841F951FA01D08958F921F
:104D00009F92AF92BF92CF92DF92EF92FF92CF939A
:104D1000DF93EC01688179818A819B81611571053E
:104D20008105910521F464E279ED8BE597E02DE1B1
:104D300033EF41E050E00E94F12649015A019B0106
:104D4000AC01A7EAB1E40E9410276B017C01ACEE34
:104D5000B4EFA50194010E941E27DC01CB018C0D4C
:104D60009D1DAE1DBF1DB7FF03C00197A109B0482F
:104D700088839983AA83BB839F77DF91CF91FF902C
:104D8000EF90DF90CF90BF90AF909F908F9008955D
:104D90000E947F26089583E191E00E947F26089576
:104DA000A0E0B0E08093130190931401A09315014B
:104DB000B09316010895F999FECF92BD81BDF89A7E
:104DC000992780B50895262FF999FECF1FBA92BD75
:104DD00081BD20BD0FB6F894FA9AF99A0FBE0196DC
:104DE0000895052E97FB1EF400940E94082757FD96
:104DF00007D00E94232707FC03D04EF40C94082709
:104E000050954095309521953F4F4F4F5F4F0895F6
:104E100090958095709561957F4F8F4F9F4F089526
:104E20000E944527A59F900DB49F900DA49F800DD3
:104E3000911D11240895B7FF0C9410270E9410278C
:104E4000821B930B0895A1E21A2EAA1BBB1BFD0126
:104E50000DC0AA1FBB1FEE1FFF1FA217B307E40759
:104E6000F50720F0A21BB30BE40BF50B661F771FB1
:104E7000881F991F1A9469F7609570958095909591
:104E80009B01AC01BD01CF010895A29FB001B39F6A
:104E9000C001A39F700D811D1124911DB29F700D43
:104EA000811D1124911D08952F923F924F925F9280
:104EB0006F927F928F929F92AF92BF92CF92DF922A
:104EC000EF92FF920F931F93CF93DF93CDB7DEB78F
:104ED000CA1BDB0B0FB6F894DEBF0FBECDBF099423
:104EE0002A88398848885F846E847D848C849B847A
:104EF000AA84B984C884DF80EE80FD800C811B8188
:104F0000AA81B981CE0FD11D0FB6F894DEBF0FBEB6
:0A4F1000CDBFED010895F894FFCF26
:104F1A008000010114000100E1000000000000FF10
:104F2A00FFFFFF010000000100000000000000AFC9
:104F3A000E240FF617D00EEE0EC50E00000000B6B6
:104F4A00167A1200C18081000000312E31202D20F6
:104F5A00406372616974004A6F6E617468616E20A1
:104F6A00486F6C6D65730053434F5245002B25649F
:104F7A0021002B256400594F55004449454421001E
:104F8A0047414D45204F564552004849474820530E
:0A4F9A00434F52453A202564000001
:00000001FF
